 gc

 Timestamp is dc667cef (reproducible build file hash)

 Preferred load address is 0000000180000000

 Start         Length     Name                   Class
 0001:00000000 00002cf0H .text$mn                CODE
 0001:00002cf0 00000036H .text$mn$00             CODE
 0001:00002d26 00000092H .text$x                 CODE
 0002:00000000 00000198H .idata$5                DATA
 0002:00000198 00000038H .00cfg                  DATA
 0002:000001d0 00000008H .CRT$XCA                DATA
 0002:000001d8 00000008H .CRT$XCZ                DATA
 0002:000001e0 00000008H .CRT$XIA                DATA
 0002:000001e8 00000008H .CRT$XIC                DATA
 0002:000001f0 00000008H .CRT$XIZ                DATA
 0002:000001f8 00000008H .CRT$XLA                DATA
 0002:00000200 00000008H .CRT$XLZ                DATA
 0002:00000208 00000008H .CRT$XPA                DATA
 0002:00000210 00000008H .CRT$XPZ                DATA
 0002:00000218 00000008H .CRT$XTA                DATA
 0002:00000220 00000010H .CRT$XTZ                DATA
 0002:00000228 00000000H .gehcont$y              DATA
 0002:00000228 00000000H .gfids$y                DATA
 0002:00000230 00001cd0H .rdata                  DATA
 0002:00001f00 00000000H .rdata$CastGuardVftablesA DATA
 0002:00001f00 00000000H .rdata$CastGuardVftablesC DATA
 0002:00001f00 00000028H .rdata$T                DATA
 0002:00001f28 000000a4H .rdata$voltmd           DATA
 0002:00001fcc 00000314H .rdata$zzzdbg           DATA
 0002:000022e0 00000008H .rtc$IAA                DATA
 0002:000022e8 00000008H .rtc$IZZ                DATA
 0002:000022f0 00000008H .rtc$TAA                DATA
 0002:000022f8 00000008H .rtc$TZZ                DATA
 0002:00002300 00000004H .tls                    DATA
 0002:00002304 00000004H .tls$                   DATA
 0002:00002308 00000008H .tls$ZZZ                DATA
 0002:00002310 000002e0H .xdata                  DATA
 0002:000025f0 00000494H .edata                  DATA
 0002:00002a84 00000064H .idata$2                DATA
 0002:00002ae8 00000018H .idata$3                DATA
 0002:00002b00 00000198H .idata$4                DATA
 0002:00002c98 0000041eH .idata$6                DATA
 0003:00000000 00000080H .data                   DATA
 0003:00000080 0001b3d8H .bss                    DATA
 0004:00000000 000003b4H .pdata                  DATA

  Address         Publics by Value              Rva+Base               Lib:Object

 0000:00000000       __AbsoluteZero             0000000000000000     <absolute>
 0000:00000000       ___safe_se_handler_count   0000000000000000     <absolute>
 0000:00000000       ___safe_se_handler_table   0000000000000000     <absolute>
 0000:00000000       __arm64x_extra_rfe_table   0000000000000000     <absolute>
 0000:00000000       __arm64x_extra_rfe_table_size 0000000000000000     <absolute>
 0000:00000000       __arm64x_native_entrypoint 0000000000000000     <absolute>
 0000:00000000       __arm64x_redirection_metadata 0000000000000000     <absolute>
 0000:00000000       __arm64x_redirection_metadata_count 0000000000000000     <absolute>
 0000:00000000       __dynamic_value_reloc_table 0000000000000000     <absolute>
 0000:00000000       __enclave_config           0000000000000000     <absolute>
 0000:00000000       __guard_check_icall_a64n_fptr 0000000000000000     <absolute>
 0000:00000000       __guard_eh_cont_count      0000000000000000     <absolute>
 0000:00000000       __guard_eh_cont_table      0000000000000000     <absolute>
 0000:00000000       __guard_fids_count         0000000000000000     <absolute>
 0000:00000000       __guard_fids_table         0000000000000000     <absolute>
 0000:00000000       __guard_iat_count          0000000000000000     <absolute>
 0000:00000000       __guard_iat_table          0000000000000000     <absolute>
 0000:00000000       __guard_longjmp_count      0000000000000000     <absolute>
 0000:00000000       __guard_longjmp_table      0000000000000000     <absolute>
 0000:00000000       __hybrid_auxiliary_iat     0000000000000000     <absolute>
 0000:00000000       __hybrid_auxiliary_iat_copy 0000000000000000     <absolute>
 0000:00000000       __hybrid_code_map          0000000000000000     <absolute>
 0000:00000000       __hybrid_code_map_count    0000000000000000     <absolute>
 0000:00000000       __x64_code_ranges_to_entry_points 0000000000000000     <absolute>
 0000:00000000       __x64_code_ranges_to_entry_points_count 0000000000000000     <absolute>
 0000:00000100       __guard_flags              0000000000000100     <absolute>
 0000:00000000       __ImageBase                0000000180000000     <linker-defined>
 0001:00000000       ?NewObject@JNIEnv_@@QEAAPEAV_jobject@@PEAV_jclass@@PEAU_jmethodID@@ZZ 0000000180001000 f i libgc.obj
 0001:00000028       ?SetEventNotificationMode@_jvmtiEnv@@QEAA?AW4jvmtiError@@W4jvmtiEventMode@@W4jvmtiEvent@@PEAV_jobject@@ZZ 0000000180001028 f i libgc.obj
 0001:00000034       ?TranslateError@@YAPEBDW4jvmtiError@@@Z 0000000180001034 f   libgc.obj
 0001:000002ec       ?nsk_jni_check_exception@@YAHPEAUJNIEnv_@@QEBDH@Z 00000001800012ec f   libgc.obj
 0001:00000430       ?nsk_jni_lverify@@YAHHPEAUJNIEnv_@@HQEBDH1ZZ 0000000180001430 f   libgc.obj
 0001:000004d0       Agent_Initialize           00000001800014d0 f   libgc.obj
 0001:000006c0       Agent_OnAttach             00000001800016c0 f   libgc.obj
 0001:000006c0       Agent_OnLoad               00000001800016c0 f   libgc.obj
 0001:000006c8       Java_nsk_jvmti_unit_FollowReferences_FollowRefObjects_addRefToVerify 00000001800016c8 f   libgc.obj
 0001:000008a0       Java_nsk_jvmti_unit_FollowReferences_FollowRefObjects_getTag 00000001800018a0 f   libgc.obj
 0001:00000960       Java_nsk_jvmti_unit_FollowReferences_FollowRefObjects_resetRefsToVerify 0000000180001960 f   libgc.obj
 0001:00000968       Java_nsk_jvmti_unit_FollowReferences_FollowRefObjects_resetTags 0000000180001968 f   libgc.obj
 0001:000009ac       Java_nsk_jvmti_unit_FollowReferences_FollowRefObjects_setTag 00000001800019ac f   libgc.obj
 0001:00000c04       Java_nsk_jvmti_unit_functions_ForceGarbageCollection_gc_GetResult 0000000180001c04 f   libgc.obj
 0001:00000c0c       Java_nsk_jvmti_unit_functions_ForceGarbageCollection_gc_checkGCFinish 0000000180001c0c f   libgc.obj
 0001:00000c34       Java_nsk_jvmti_unit_functions_ForceGarbageCollection_gc_checkGCStart 0000000180001c34 f   libgc.obj
 0001:00000c5c       Java_nsk_jvmti_unit_functions_ForceGarbageCollection_gc_jvmtiForceGC 0000000180001c5c f   libgc.obj
 0001:00000ca0       Java_nsk_share_jvmti_ArgumentHandler_getAgentOptionsString 0000000180001ca0 f   libgc.obj
 0001:00000d50       Java_nsk_share_jvmti_DebugeeClass_checkStatus 0000000180001d50 f   libgc.obj
 0001:00000dd8       Java_nsk_share_jvmti_DebugeeClass_resetAgentData 0000000180001dd8 f   libgc.obj
 0001:00000e38       Java_nsk_share_jvmti_RedefineAgent_agentStatus 0000000180001e38 f   libgc.obj
 0001:00000e44       Java_nsk_share_jvmti_RedefineAgent_isRedefined 0000000180001e44 f   libgc.obj
 0001:00000e50       Java_nsk_share_jvmti_RedefineAgent_redefineAttempted 0000000180001e50 f   libgc.obj
 0001:00000e5c       MA_checkStatus             0000000180001e5c f   libgc.obj
 0001:00000f00       __local_stdio_printf_options 0000000180001f00 f i libgc.obj
 0001:000010e0       debug_printf               00000001800020e0 f   libgc.obj
 0001:0000113c       exitOnError                000000018000213c f   libgc.obj
 0001:000011f0       fprintf                    00000001800021f0 f i libgc.obj
 0001:00001234       gc_finish                  0000000180002234 f   libgc.obj
 0001:00001248       gc_start                   0000000180002248 f   libgc.obj
 0001:0000125c       init_callbacks             000000018000225c f   libgc.obj
 0001:000012b4       nsk_jvmti_lverify          00000001800022b4 f   libgc.obj
 0001:000013a4       nsk_jvmti_resetAgentData   00000001800023a4 f   libgc.obj
 0001:00001424       nsk_jvmti_setFailStatus    0000000180002424 f   libgc.obj
 0001:00001460       nsk_lcomplain              0000000180002460 f   libgc.obj
 0001:00001480       nsk_ldisplay               0000000180002480 f   libgc.obj
 0001:000014a0       nsk_ltrace                 00000001800024a0 f   libgc.obj
 0001:000014c0       nsk_lvcomplain             00000001800024c0 f   libgc.obj
 0001:00001678       nsk_lvdisplay              0000000180002678 f   libgc.obj
 0001:000016c4       nsk_lverify                00000001800026c4 f   libgc.obj
 0001:00001720       nsk_lvtrace                0000000180002720 f   libgc.obj
 0001:00001780       nsk_printf                 0000000180002780 f   libgc.obj
 0001:000017a8       nsk_vprintf                00000001800027a8 f   libgc.obj
 0001:0000185c       printf                     000000018000285c f i libgc.obj
 0001:00001d84       vmExit                     0000000180002d84 f   libgc.obj
 0001:00001dbc       vmInit                     0000000180002dbc f   libgc.obj
 0001:00001dc8       __raise_securityfailure    0000000180002dc8 f   MSVCRT:gs_report.obj
 0001:00001dfc       __report_gsfailure         0000000180002dfc f   MSVCRT:gs_report.obj
 0001:0000203c       __GSHandlerCheck           000000018000303c f   MSVCRT:gshandler.obj
 0001:0000205c       __GSHandlerCheckCommon     000000018000305c f   MSVCRT:gshandler.obj
 0001:000020d0       __security_check_cookie    00000001800030d0 f   MSVCRT:amdsecgs.obj
 0001:00002410       _DllMainCRTStartup         0000000180003410 f   MSVCRT:dll_dllmain.obj
 0001:00002450       __scrt_acquire_startup_lock 0000000180003450 f   MSVCRT:utility.obj
 0001:0000248c       __scrt_dllmain_after_initialize_c 000000018000348c f   MSVCRT:utility.obj
 0001:000024c0       __scrt_dllmain_before_initialize_c 00000001800034c0 f   MSVCRT:utility.obj
 0001:000024d8       __scrt_dllmain_crt_thread_attach 00000001800034d8 f   MSVCRT:utility.obj
 0001:00002500       __scrt_dllmain_crt_thread_detach 0000000180003500 f   MSVCRT:utility.obj
 0001:00002518       __scrt_dllmain_exception_filter 0000000180003518 f   MSVCRT:utility.obj
 0001:00002578       __scrt_dllmain_uninitialize_c 0000000180003578 f   MSVCRT:utility.obj
 0001:000025a8       __scrt_dllmain_uninitialize_critical 00000001800035a8 f   MSVCRT:utility.obj
 0001:000025bc       __scrt_initialize_crt      00000001800035bc f   MSVCRT:utility.obj
 0001:00002608       __scrt_initialize_onexit_tables 0000000180003608 f   MSVCRT:utility.obj
 0001:00002694       __scrt_is_nonwritable_in_current_image 0000000180003694 f   MSVCRT:utility.obj
 0001:0000272c       __scrt_release_startup_lock 000000018000372c f   MSVCRT:utility.obj
 0001:00002750       __scrt_uninitialize_crt    0000000180003750 f   MSVCRT:utility.obj
 0001:0000277c       _onexit                    000000018000377c f   MSVCRT:utility.obj
 0001:000027b8       atexit                     00000001800037b8 f   MSVCRT:utility.obj
 0001:000027d0       __crt_debugger_hook        00000001800037d0 f   MSVCRT:utility_desktop.obj
 0001:000027d8       __scrt_fastfail            00000001800037d8 f   MSVCRT:utility_desktop.obj
 0001:00002924       _guard_check_icall_nop     0000000180003924 f i MSVCRT:guard_support.obj
 0001:00002928       __security_init_cookie     0000000180003928 f   MSVCRT:gs_support.obj
 0001:000029d4       DllMain                    00000001800039d4 f   MSVCRT:dll_dllmain_stub.obj
 0001:000029f8       ?__scrt_initialize_type_info@@YAXXZ 00000001800039f8 f   MSVCRT:tncleanup.obj
 0001:00002a08       ?__scrt_uninitialize_type_info@@YAXXZ 0000000180003a08 f   MSVCRT:tncleanup.obj
 0001:00002a14       __local_stdio_scanf_options 0000000180003a14 f i MSVCRT:default_local_stdio_options.obj
 0001:00002a1c       __scrt_initialize_default_local_stdio_options 0000000180003a1c f   MSVCRT:default_local_stdio_options.obj
 0001:00002a38       __scrt_get_dyn_tls_init_callback 0000000180003a38 f   MSVCRT:dyn_tls_init.obj
 0001:00002a40       _RTC_Initialize            0000000180003a40 f   MSVCRT:initsect.obj
 0001:00002a7c       _RTC_Terminate             0000000180003a7c f   MSVCRT:initsect.obj
 0001:00002ab8       __isa_available_init       0000000180003ab8 f   MSVCRT:cpu_disp.obj
 0001:00002c64       _get_startup_argv_mode     0000000180003c64 f   MSVCRT:argv_mode.obj
 0001:00002c6c       __scrt_is_ucrt_dll_in_use  0000000180003c6c f   MSVCRT:ucrt_detection.obj
 0001:00002c80       memcpy                     0000000180003c80 f   vcruntime:VCRUNTIME140.dll
 0001:00002c86       memset                     0000000180003c86 f   vcruntime:VCRUNTIME140.dll
 0001:00002c8c       strchr                     0000000180003c8c f   vcruntime:VCRUNTIME140.dll
 0001:00002c92       strstr                     0000000180003c92 f   vcruntime:VCRUNTIME140.dll
 0001:00002c98       __C_specific_handler       0000000180003c98 f   vcruntime:VCRUNTIME140.dll
 0001:00002c9e       __std_type_info_destroy_list 0000000180003c9e f   vcruntime:VCRUNTIME140.dll
 0001:00002ca4       strlen                     0000000180003ca4 f   ucrt:api-ms-win-crt-string-l1-1-0.dll
 0001:00002caa       _initterm                  0000000180003caa f   ucrt:api-ms-win-crt-runtime-l1-1-0.dll
 0001:00002cb0       _initterm_e                0000000180003cb0 f   ucrt:api-ms-win-crt-runtime-l1-1-0.dll
 0001:00002cb6       _seh_filter_dll            0000000180003cb6 f   ucrt:api-ms-win-crt-runtime-l1-1-0.dll
 0001:00002cbc       _configure_narrow_argv     0000000180003cbc f   ucrt:api-ms-win-crt-runtime-l1-1-0.dll
 0001:00002cc2       _initialize_narrow_environment 0000000180003cc2 f   ucrt:api-ms-win-crt-runtime-l1-1-0.dll
 0001:00002cc8       _initialize_onexit_table   0000000180003cc8 f   ucrt:api-ms-win-crt-runtime-l1-1-0.dll
 0001:00002cce       _register_onexit_function  0000000180003cce f   ucrt:api-ms-win-crt-runtime-l1-1-0.dll
 0001:00002cd4       _execute_onexit_table      0000000180003cd4 f   ucrt:api-ms-win-crt-runtime-l1-1-0.dll
 0001:00002cda       _crt_atexit                0000000180003cda f   ucrt:api-ms-win-crt-runtime-l1-1-0.dll
 0001:00002ce0       _cexit                     0000000180003ce0 f   ucrt:api-ms-win-crt-runtime-l1-1-0.dll
 0001:00002ce8       __acrt_initialize          0000000180003ce8 f   MSVCRT:ucrt_stubs.obj
 0001:00002ce8       __acrt_thread_attach       0000000180003ce8 f   MSVCRT:ucrt_stubs.obj
 0001:00002ce8       __acrt_thread_detach       0000000180003ce8 f   MSVCRT:ucrt_stubs.obj
 0001:00002ce8       __acrt_uninitialize        0000000180003ce8 f   MSVCRT:ucrt_stubs.obj
 0001:00002ce8       __acrt_uninitialize_critical 0000000180003ce8 f   MSVCRT:ucrt_stubs.obj
 0001:00002ce8       __scrt_stub_for_acrt_initialize 0000000180003ce8 f   MSVCRT:ucrt_stubs.obj
 0001:00002ce8       __scrt_stub_for_acrt_thread_attach 0000000180003ce8 f   MSVCRT:ucrt_stubs.obj
 0001:00002ce8       __scrt_stub_for_acrt_thread_detach 0000000180003ce8 f   MSVCRT:ucrt_stubs.obj
 0001:00002ce8       __scrt_stub_for_acrt_uninitialize 0000000180003ce8 f   MSVCRT:ucrt_stubs.obj
 0001:00002ce8       __scrt_stub_for_acrt_uninitialize_critical 0000000180003ce8 f   MSVCRT:ucrt_stubs.obj
 0001:00002ce8       __vcrt_initialize          0000000180003ce8 f   MSVCRT:ucrt_stubs.obj
 0001:00002ce8       __vcrt_thread_attach       0000000180003ce8 f   MSVCRT:ucrt_stubs.obj
 0001:00002ce8       __vcrt_thread_detach       0000000180003ce8 f   MSVCRT:ucrt_stubs.obj
 0001:00002ce8       __vcrt_uninitialize        0000000180003ce8 f   MSVCRT:ucrt_stubs.obj
 0001:00002ce8       __vcrt_uninitialize_critical 0000000180003ce8 f   MSVCRT:ucrt_stubs.obj
 0001:00002cec       __scrt_stub_for_is_c_termination_complete 0000000180003cec f   MSVCRT:ucrt_stubs.obj
 0001:00002cec       _is_c_termination_complete 0000000180003cec f   MSVCRT:ucrt_stubs.obj
 0001:00002d00       _guard_dispatch_icall_nop  0000000180003d00 f   MSVCRT:guard_dispatch.obj
 0001:00002d20       _guard_xfg_dispatch_icall_nop 0000000180003d20 f   MSVCRT:guard_xfg_dispatch.obj
 0002:00000000       __imp_RtlCaptureContext    0000000180004000     kernel32:KERNEL32.dll
 0002:00000008       __imp_RtlLookupFunctionEntry 0000000180004008     kernel32:KERNEL32.dll
 0002:00000010       __imp_RtlVirtualUnwind     0000000180004010     kernel32:KERNEL32.dll
 0002:00000018       __imp_UnhandledExceptionFilter 0000000180004018     kernel32:KERNEL32.dll
 0002:00000020       __imp_SetUnhandledExceptionFilter 0000000180004020     kernel32:KERNEL32.dll
 0002:00000028       __imp_GetCurrentProcess    0000000180004028     kernel32:KERNEL32.dll
 0002:00000030       __imp_TerminateProcess     0000000180004030     kernel32:KERNEL32.dll
 0002:00000038       __imp_IsProcessorFeaturePresent 0000000180004038     kernel32:KERNEL32.dll
 0002:00000040       __imp_CloseHandle          0000000180004040     kernel32:KERNEL32.dll
 0002:00000048       __imp_InitializeCriticalSectionAndSpinCount 0000000180004048     kernel32:KERNEL32.dll
 0002:00000050       __imp_DeleteCriticalSection 0000000180004050     kernel32:KERNEL32.dll
 0002:00000058       __imp_CreateEventW         0000000180004058     kernel32:KERNEL32.dll
 0002:00000060       __imp_GetModuleHandleW     0000000180004060     kernel32:KERNEL32.dll
 0002:00000068       __imp_GetProcAddress       0000000180004068     kernel32:KERNEL32.dll
 0002:00000070       __imp_IsDebuggerPresent    0000000180004070     kernel32:KERNEL32.dll
 0002:00000078       __imp_QueryPerformanceCounter 0000000180004078     kernel32:KERNEL32.dll
 0002:00000080       __imp_GetCurrentProcessId  0000000180004080     kernel32:KERNEL32.dll
 0002:00000088       __imp_GetCurrentThreadId   0000000180004088     kernel32:KERNEL32.dll
 0002:00000090       __imp_GetSystemTimeAsFileTime 0000000180004090     kernel32:KERNEL32.dll
 0002:00000098       __imp_DisableThreadLibraryCalls 0000000180004098     kernel32:KERNEL32.dll
 0002:000000a0       __imp_InitializeSListHead  00000001800040a0     kernel32:KERNEL32.dll
 0002:000000a8       \177KERNEL32_NULL_THUNK_DATA 00000001800040a8     kernel32:KERNEL32.dll
 0002:000000b0       __imp_memcpy               00000001800040b0     vcruntime:VCRUNTIME140.dll
 0002:000000b8       __imp_memset               00000001800040b8     vcruntime:VCRUNTIME140.dll
 0002:000000c0       __imp_strchr               00000001800040c0     vcruntime:VCRUNTIME140.dll
 0002:000000c8       __imp_strstr               00000001800040c8     vcruntime:VCRUNTIME140.dll
 0002:000000d0       __imp___C_specific_handler 00000001800040d0     vcruntime:VCRUNTIME140.dll
 0002:000000d8       __imp___std_type_info_destroy_list 00000001800040d8     vcruntime:VCRUNTIME140.dll
 0002:000000e0       \177VCRUNTIME140_NULL_THUNK_DATA 00000001800040e0     vcruntime:VCRUNTIME140.dll
 0002:000000e8       __imp__errno               00000001800040e8     ucrt:api-ms-win-crt-runtime-l1-1-0.dll
 0002:000000f0       __imp_exit                 00000001800040f0     ucrt:api-ms-win-crt-runtime-l1-1-0.dll
 0002:000000f8       __imp__cexit               00000001800040f8     ucrt:api-ms-win-crt-runtime-l1-1-0.dll
 0002:00000100       __imp__crt_atexit          0000000180004100     ucrt:api-ms-win-crt-runtime-l1-1-0.dll
 0002:00000108       __imp__execute_onexit_table 0000000180004108     ucrt:api-ms-win-crt-runtime-l1-1-0.dll
 0002:00000110       __imp__register_onexit_function 0000000180004110     ucrt:api-ms-win-crt-runtime-l1-1-0.dll
 0002:00000118       __imp__initialize_onexit_table 0000000180004118     ucrt:api-ms-win-crt-runtime-l1-1-0.dll
 0002:00000120       __imp__initialize_narrow_environment 0000000180004120     ucrt:api-ms-win-crt-runtime-l1-1-0.dll
 0002:00000128       __imp__configure_narrow_argv 0000000180004128     ucrt:api-ms-win-crt-runtime-l1-1-0.dll
 0002:00000130       __imp__seh_filter_dll      0000000180004130     ucrt:api-ms-win-crt-runtime-l1-1-0.dll
 0002:00000138       __imp__initterm_e          0000000180004138     ucrt:api-ms-win-crt-runtime-l1-1-0.dll
 0002:00000140       __imp__initterm            0000000180004140     ucrt:api-ms-win-crt-runtime-l1-1-0.dll
 0002:00000148       \177api-ms-win-crt-runtime-l1-1-0_NULL_THUNK_DATA 0000000180004148     ucrt:api-ms-win-crt-runtime-l1-1-0.dll
 0002:00000150       __imp___acrt_iob_func      0000000180004150     ucrt:api-ms-win-crt-stdio-l1-1-0.dll
 0002:00000158       __imp_fflush               0000000180004158     ucrt:api-ms-win-crt-stdio-l1-1-0.dll
 0002:00000160       __imp___stdio_common_vsprintf 0000000180004160     ucrt:api-ms-win-crt-stdio-l1-1-0.dll
 0002:00000168       __imp___stdio_common_vfprintf 0000000180004168     ucrt:api-ms-win-crt-stdio-l1-1-0.dll
 0002:00000170       \177api-ms-win-crt-stdio-l1-1-0_NULL_THUNK_DATA 0000000180004170     ucrt:api-ms-win-crt-stdio-l1-1-0.dll
 0002:00000178       __imp__strdup              0000000180004178     ucrt:api-ms-win-crt-string-l1-1-0.dll
 0002:00000178       __imp_strdup               0000000180004178     ucrt:api-ms-win-crt-string-l1-1-0.dll
 0002:00000180       __imp_strlen               0000000180004180     ucrt:api-ms-win-crt-string-l1-1-0.dll
 0002:00000188       __imp_strncpy              0000000180004188     ucrt:api-ms-win-crt-string-l1-1-0.dll
 0002:00000190       \177api-ms-win-crt-string-l1-1-0_NULL_THUNK_DATA 0000000180004190     ucrt:api-ms-win-crt-string-l1-1-0.dll
 0002:00000198       __guard_check_icall_fptr   0000000180004198     MSVCRT:guard_support.obj
 0002:000001a0       __guard_xfg_check_icall_fptr 00000001800041a0     MSVCRT:guard_support.obj
 0002:000001a8       __guard_dispatch_icall_fptr 00000001800041a8     MSVCRT:guard_support.obj
 0002:000001b0       __guard_xfg_dispatch_icall_fptr 00000001800041b0     MSVCRT:guard_support.obj
 0002:000001b8       __guard_xfg_table_dispatch_icall_fptr 00000001800041b8     MSVCRT:guard_support.obj
 0002:000001c0       __castguard_check_failure_os_handled_fptr 00000001800041c0     MSVCRT:guard_support.obj
 0002:000001c8       __guard_memcpy_fptr        00000001800041c8     vcruntime:softmemtag.obj
 0002:000001d0       __xc_a                     00000001800041d0     MSVCRT:initializers.obj
 0002:000001d8       __xc_z                     00000001800041d8     MSVCRT:initializers.obj
 0002:000001e0       __xi_a                     00000001800041e0     MSVCRT:initializers.obj
 0002:000001f0       __xi_z                     00000001800041f0     MSVCRT:initializers.obj
 0002:000001f8       __xl_a                     00000001800041f8     MSVCRT:tlssup.obj
 0002:00000200       __xl_z                     0000000180004200     MSVCRT:tlssup.obj
 0002:00000208       __xp_a                     0000000180004208     MSVCRT:initializers.obj
 0002:00000210       __xp_z                     0000000180004210     MSVCRT:initializers.obj
 0002:00000218       __xt_a                     0000000180004218     MSVCRT:initializers.obj
 0002:00000220       __xt_z                     0000000180004220     MSVCRT:initializers.obj
 0002:00000230       g_refKindStr               0000000180004230     libgc.obj
 0002:000003e0       ??_C@_09BPLDFGCI@unknown_0@ 00000001800043e0     libgc.obj
 0002:000003f0       ??_C@_0BL@FPNMECJD@JVMTI_HEAP_REFERENCE_CLASS@ 00000001800043f0     libgc.obj
 0002:00000410       ??_C@_0BL@FKGKKLNM@JVMTI_HEAP_REFERENCE_FIELD@ 0000000180004410     libgc.obj
 0002:00000430       ??_C@_0CD@CAEHCFJF@JVMTI_HEAP_REFERENCE_ARRAY_ELEM@ 0000000180004430     libgc.obj
 0002:00000458       ??_C@_0CC@DNEBMCNK@JVMTI_HEAP_REFERENCE_CLASS_LOAD@ 0000000180004458     libgc.obj
 0002:00000480       ??_C@_0BN@CJMIPEBB@JVMTI_HEAP_REFERENCE_SIGNERS@ 0000000180004480     libgc.obj
 0002:000004a0       ??_C@_0CH@HBOIDPEB@JVMTI_HEAP_REFERENCE_PROTECTION@ 00000001800044a0     libgc.obj
 0002:000004c8       ??_C@_0BP@MDKGDGKL@JVMTI_HEAP_REFERENCE_INTERFACE@ 00000001800044c8     libgc.obj
 0002:000004e8       ??_C@_0CC@JJMIHNJH@JVMTI_HEAP_REFERENCE_STATIC_FIE@ 00000001800044e8     libgc.obj
 0002:00000510       ??_C@_0CD@IDHEEGID@JVMTI_HEAP_REFERENCE_CONSTANT_P@ 0000000180004510     libgc.obj
 0002:00000538       ??_C@_0CA@EFFCHNG@JVMTI_HEAP_REFERENCE_SUPERCLASS@ 0000000180004538     libgc.obj
 0002:00000558       ??_C@_0L@PCDFHGCJ@unknown_11@ 0000000180004558     libgc.obj
 0002:00000568       ??_C@_0L@NJBICFOK@unknown_12@ 0000000180004568     libgc.obj
 0002:00000578       ??_C@_0L@MAADBEKL@unknown_13@ 0000000180004578     libgc.obj
 0002:00000588       ??_C@_0L@IPECICGM@unknown_14@ 0000000180004588     libgc.obj
 0002:00000598       ??_C@_0L@JGFJLDCN@unknown_15@ 0000000180004598     libgc.obj
 0002:000005a8       ??_C@_0L@LNHEOAOO@unknown_16@ 00000001800045a8     libgc.obj
 0002:000005b8       ??_C@_0L@KEGPNBKP@unknown_17@ 00000001800045b8     libgc.obj
 0002:000005c8       ??_C@_0L@CDPHMNGA@unknown_18@ 00000001800045c8     libgc.obj
 0002:000005d8       ??_C@_0L@DKOMPMCB@unknown_19@ 00000001800045d8     libgc.obj
 0002:000005e8       ??_C@_0L@OJGIPJDB@unknown_20@ 00000001800045e8     libgc.obj
 0002:000005f8       ??_C@_0CA@KAOFNDEM@JVMTI_HEAP_REFERENCE_JNI_GLOBAL@ 00000001800045f8     libgc.obj
 0002:00000618       ??_C@_0CC@HPFAJBK@JVMTI_HEAP_REFERENCE_SYSTEM_CLA@ 0000000180004618     libgc.obj
 0002:00000640       ??_C@_0BN@FDEGFOHC@JVMTI_HEAP_REFERENCE_MONITOR@ 0000000180004640     libgc.obj
 0002:00000660       ??_C@_0CB@HKIBCMAJ@JVMTI_HEAP_REFERENCE_STACK_LOCA@ 0000000180004660     libgc.obj
 0002:00000688       ??_C@_0BP@EAACMMOE@JVMTI_HEAP_REFERENCE_JNI_LOCAL@ 0000000180004688     libgc.obj
 0002:000006a8       ??_C@_0BM@IJDEOGOE@JVMTI_HEAP_REFERENCE_THREAD@ 00000001800046a8     libgc.obj
 0002:000006c8       ??_C@_0BL@EDGPPKC@JVMTI_HEAP_REFERENCE_OTHER@ 00000001800046c8     libgc.obj
 0002:000006e4       ??_C@_04BCJPDBDA@Code@     00000001800046e4     libgc.obj
 0002:000006f0       ??_C@_0BA@OCLMCFKC@LineNumberTable@ 00000001800046f0     libgc.obj
 0002:00000700       ??_C@_0BD@CPAEPILC@LocalVariableTable@ 0000000180004700     libgc.obj
 0002:00000718       ??_C@_0BH@NMBDNHBD@LocalVariableTypeTable@ 0000000180004718     libgc.obj
 0002:00000730       ??_C@_0O@HIHEEDNJ@StackMapTable@ 0000000180004730     libgc.obj
 0002:00000740       ??_C@_0L@HCDIAMJG@?9?5?$CFs?0?5?$CFd?3?5@ 0000000180004740     libgc.obj
 0002:00000750       ??_C@_0JI@HLPECLFI@?$CD?5?4?4?4?6?$CD?5ERROR?3?5too?5many?5complai@ 0000000180004750     libgc.obj
 0002:000007f0       ??_C@_0ED@JNEKCCOB@The?5following?5fake?5exception?5st@ 00000001800047f0     libgc.obj
 0002:00000838       ??_C@_0CN@FCNMDFBH@nsk?4share?4Fake_Exception_for_RU@ 0000000180004838     libgc.obj
 0002:00000868       ??_C@_08PGFFNAEI@?$CI?$CFs?3?$CFd?$CJ?5@ 0000000180004868     libgc.obj
 0002:00000878       ??_C@_0DP@IENMAEGI@s?2test?2hotspot?2jtreg?2vmTestbase@ 0000000180004878     libgc.obj
 0002:000008b8       ??_C@_0BL@NDJLFFJB@?7at?5nsk_lvcomplain?$CI?$CFs?3?$CFd?$CJ?6@ 00000001800048b8     libgc.obj
 0002:000008d8       ??_C@_0BC@JOOKAFKF@?$CD?5ERROR?3?5?$CFs?0?5?$CFd?3?5@ 00000001800048d8     libgc.obj
 0002:000008f0       ??_C@_09KJEAHMEH@?$CD?5ERROR?3?5@ 00000001800048f0     libgc.obj
 0002:000008fc       ??_C@_02GPIOPFAK@?$DO?$DO@ 00000001800048fc     libgc.obj
 0002:00000900       ??_C@_02FODMEDOG@?$DM?$DM@ 0000000180004900     libgc.obj
 0002:00000904       ??_C@_02DJGKEECL@?4?4@     0000000180004904     libgc.obj
 0002:00000908       ??_C@_0O@CJPGJOAF@?9?5?$CFs?0?5?$CFd?3?5?$CFs?5@ 0000000180004908     libgc.obj
 0002:00000918       ??_C@_0CB@IAKPDOIC@?$CD?5?5?5verified?5assertion?5is?5FALSE@ 0000000180004918     libgc.obj
 0002:00000940       ??_C@_0CO@LGONDEPD@stdout?3?5fflush?5failed?5?9?5err?$DN?$CFd?5@ 0000000180004940     libgc.obj
 0002:00000970       ??_C@_0CO@KBGKJPBD@stderr?3?5fflush?5failed?5?9?5err?$DN?$CFd?5@ 0000000180004970     libgc.obj
 0002:000009a0       ??_C@_0BB@JCNMKLLK@JVMTI_ERROR_NONE@ 00000001800049a0     libgc.obj
 0002:000009b8       ??_C@_0BL@LDIMKLPH@JVMTI_ERROR_INVALID_THREAD@ 00000001800049b8     libgc.obj
 0002:000009d8       ??_C@_0CB@PJFPAIKJ@JVMTI_ERROR_INVALID_THREAD_GROU@ 00000001800049d8     libgc.obj
 0002:00000a00       ??_C@_0BN@LLMKHMNF@JVMTI_ERROR_INVALID_PRIORITY@ 0000000180004a00     libgc.obj
 0002:00000a20       ??_C@_0CB@MBOFKAGB@JVMTI_ERROR_THREAD_NOT_SUSPENDE@ 0000000180004a20     libgc.obj
 0002:00000a48       ??_C@_0BN@FABOLPBI@JVMTI_ERROR_THREAD_SUSPENDED@ 0000000180004a48     libgc.obj
 0002:00000a68       ??_C@_0BN@FDGNOBJM@JVMTI_ERROR_THREAD_NOT_ALIVE@ 0000000180004a68     libgc.obj
 0002:00000a88       ??_C@_0BL@GOBIFKNJ@JVMTI_ERROR_INVALID_OBJECT@ 0000000180004a88     libgc.obj
 0002:00000aa8       ??_C@_0BK@FCMAJPPC@JVMTI_ERROR_INVALID_CLASS@ 0000000180004aa8     libgc.obj
 0002:00000ac8       ??_C@_0BP@IKLLBKEB@JVMTI_ERROR_CLASS_NOT_PREPARED@ 0000000180004ac8     libgc.obj
 0002:00000ae8       ??_C@_0BN@KLPPLKG@JVMTI_ERROR_INVALID_METHODID@ 0000000180004ae8     libgc.obj
 0002:00000b08       ??_C@_0BN@BCEKOKND@JVMTI_ERROR_INVALID_LOCATION@ 0000000180004b08     libgc.obj
 0002:00000b28       ??_C@_0BM@DFDGPME@JVMTI_ERROR_INVALID_FIELDID@ 0000000180004b28     libgc.obj
 0002:00000b48       ??_C@_0BL@NELIEPEC@JVMTI_ERROR_NO_MORE_FRAMES@ 0000000180004b48     libgc.obj
 0002:00000b68       ??_C@_0BJ@BDBECFDM@JVMTI_ERROR_OPAQUE_FRAME@ 0000000180004b68     libgc.obj
 0002:00000b88       ??_C@_0BK@MIIFNLOB@JVMTI_ERROR_TYPE_MISMATCH@ 0000000180004b88     libgc.obj
 0002:00000ba8       ??_C@_0BJ@HPCAOILC@JVMTI_ERROR_INVALID_SLOT@ 0000000180004ba8     libgc.obj
 0002:00000bc8       ??_C@_0BG@CHILOPNI@JVMTI_ERROR_DUPLICATE@ 0000000180004bc8     libgc.obj
 0002:00000be0       ??_C@_0BG@DIEMLHKM@JVMTI_ERROR_NOT_FOUND@ 0000000180004be0     libgc.obj
 0002:00000bf8       ??_C@_0BM@NHMCKHOB@JVMTI_ERROR_INVALID_MONITOR@ 0000000180004bf8     libgc.obj
 0002:00000c18       ??_C@_0BO@PPEDAJGL@JVMTI_ERROR_NOT_MONITOR_OWNER@ 0000000180004c18     libgc.obj
 0002:00000c38       ??_C@_0BG@FCAIPEID@JVMTI_ERROR_INTERRUPT@ 0000000180004c38     libgc.obj
 0002:00000c50       ??_C@_0CB@EGDBNKOI@JVMTI_ERROR_INVALID_CLASS_FORMA@ 0000000180004c50     libgc.obj
 0002:00000c78       ??_C@_0CG@DGKOGIAL@JVMTI_ERROR_CIRCULAR_CLASS_DEFI@ 0000000180004c78     libgc.obj
 0002:00000ca0       ??_C@_0BP@ICEALPKC@JVMTI_ERROR_FAILS_VERIFICATION@ 0000000180004ca0     libgc.obj
 0002:00000cc0       ??_C@_0DC@JDACLMIO@JVMTI_ERROR_UNSUPPORTED_REDEFIN@ 0000000180004cc0     libgc.obj
 0002:00000cf8       ??_C@_0DE@GKDKNOMJ@JVMTI_ERROR_UNSUPPORTED_REDEFIN@ 0000000180004cf8     libgc.obj
 0002:00000d30       ??_C@_0BO@LAFKIOG@JVMTI_ERROR_INVALID_TYPESTATE@ 0000000180004d30     libgc.obj
 0002:00000d50       ??_C@_0DH@INDGCLLB@JVMTI_ERROR_UNSUPPORTED_REDEFIN@ 0000000180004d50     libgc.obj
 0002:00000d88       ??_C@_0DE@NHEOMMGI@JVMTI_ERROR_UNSUPPORTED_REDEFIN@ 0000000180004d88     libgc.obj
 0002:00000dc0       ??_C@_0CA@EKPNJOEP@JVMTI_ERROR_UNSUPPORTED_VERSION@ 0000000180004dc0     libgc.obj
 0002:00000de0       ??_C@_0BN@OFFMAHHL@JVMTI_ERROR_NAMES_DONT_MATCH@ 0000000180004de0     libgc.obj
 0002:00000e00       ??_C@_0DN@HHBBLAKE@JVMTI_ERROR_UNSUPPORTED_REDEFIN@ 0000000180004e00     libgc.obj
 0002:00000e40       ??_C@_0DO@HMBGBGNA@JVMTI_ERROR_UNSUPPORTED_REDEFIN@ 0000000180004e40     libgc.obj
 0002:00000e80       ??_C@_0BP@PBECGKHJ@JVMTI_ERROR_UNMODIFIABLE_CLASS@ 0000000180004e80     libgc.obj
 0002:00000ea0       ??_C@_0BK@CANILEHF@JVMTI_ERROR_NOT_AVAILABLE@ 0000000180004ea0     libgc.obj
 0002:00000ec0       ??_C@_0CE@INJKMEFK@JVMTI_ERROR_MUST_POSSESS_CAPABI@ 0000000180004ec0     libgc.obj
 0002:00000ee8       ??_C@_0BJ@LBFPFPDM@JVMTI_ERROR_NULL_POINTER@ 0000000180004ee8     libgc.obj
 0002:00000f08       ??_C@_0BP@CHJPNNEM@JVMTI_ERROR_ABSENT_INFORMATION@ 0000000180004f08     libgc.obj
 0002:00000f28       ??_C@_0BP@OMFMNLC@JVMTI_ERROR_INVALID_EVENT_TYPE@ 0000000180004f28     libgc.obj
 0002:00000f48       ??_C@_0BN@BIBNPHHO@JVMTI_ERROR_ILLEGAL_ARGUMENT@ 0000000180004f48     libgc.obj
 0002:00000f68       ??_C@_0BK@KKNDHDCE@JVMTI_ERROR_NATIVE_METHOD@ 0000000180004f68     libgc.obj
 0002:00000f88       ??_C@_0BK@PMKCFHAE@JVMTI_ERROR_OUT_OF_MEMORY@ 0000000180004f88     libgc.obj
 0002:00000fa8       ??_C@_0BK@NNJBDMNB@JVMTI_ERROR_ACCESS_DENIED@ 0000000180004fa8     libgc.obj
 0002:00000fc8       ??_C@_0BI@GHECLMNC@JVMTI_ERROR_WRONG_PHASE@ 0000000180004fc8     libgc.obj
 0002:00000fe0       ??_C@_0BF@OLIHJOII@JVMTI_ERROR_INTERNAL@ 0000000180004fe0     libgc.obj
 0002:00000ff8       ??_C@_0BO@EOHGKJHI@JVMTI_ERROR_UNATTACHED_THREAD@ 0000000180004ff8     libgc.obj
 0002:00001018       ??_C@_0CA@LKHFDACL@JVMTI_ERROR_INVALID_ENVIRONMENT@ 0000000180005018     libgc.obj
 0002:00001038       ??_C@_0BA@MMFHLOKK@?$DMunknown?5error?$DO@ 0000000180005038     libgc.obj
 0002:00001048       ??_C@_0CF@CBHOKDB@throwable?5?$DN?5jni?9?$DOExceptionOccur@ 0000000180005048     libgc.obj
 0002:00001070       ??_C@_03OFAPEBGM@?$CFs?6@  0000000180005070     libgc.obj
 0002:00001078       ??_C@_0DM@LPIGEGNJ@s?2test?2hotspot?2jtreg?2vmTestbase@ 0000000180005078     libgc.obj
 0002:000010b8       ??_C@_0CC@NFCNPEPK@Exception?5in?5JNI?5call?5?$CIcleared?$CJ@ 00000001800050b8     libgc.obj
 0002:000010e0       ??_C@_0BJ@IBAKFIKF@jni?9?$DOExceptionDescribe?$CI?$CJ@ 00000001800050e0     libgc.obj
 0002:00001100       ??_C@_0BG@GGKALKMH@jni?9?$DOExceptionClear?$CI?$CJ@ 0000000180005100     libgc.obj
 0002:00001118       ??_C@_0CF@JMGFGJLJ@?$CD?5?5?5verified?5JNI?5assertion?5is?5F@ 0000000180005118     libgc.obj
 0002:00001140       ??_C@_0CB@MLNJNCLJ@?5?5jvmti?5error?3?5code?$DN?$CFd?0?5name?$DN?$CFs@ 0000000180005140     libgc.obj
 0002:00001168       ??_C@_0CD@OHBGDKMK@?$CD?5?5?5jvmti?5error?3?5code?$DN?$CFd?0?5name?$DN@ 0000000180005168     libgc.obj
 0002:00001190       ??_C@_0CG@JNNCGPHB@?$CD?5?5?5error?5expected?3?5code?$DN?$CFd?0?5na@ 0000000180005190     libgc.obj
 0002:000011c0       ??_C@_0EB@IMGKPCGE@?$CIstr_obj?5?$DN?5jni?9?$DONewStringUTF?$CIco@ 00000001800051c0     libgc.obj
 0002:00001210       ??_C@_0EA@HFOGGBCC@s?2test?2hotspot?2jtreg?2vmTestbase@ 0000000180005210     libgc.obj
 0002:00001250       ??_C@_05KKCIMGE@error@     0000000180005250     libgc.obj
 0002:00001258       ??_C@_0CJ@JACLEAA@Test?5failed?5by?5setFailStatus?$CI?$CJ?4@ 0000000180005258     libgc.obj
 0002:00001290       ??_C@_0EA@PNBCDMOA@s?2test?2hotspot?2jtreg?2vmTestbase@ 0000000180005290     libgc.obj
 0002:000012d0       ??_C@_0DI@ILAHDLMP@?$CI?$CKagentThreadProc?$CJ?$CIjvmti_env?0?5a@ 00000001800052d0     libgc.obj
 0002:00001308       ??_C@_0BD@KDBALNLB@JVMTI?5agent?5thread@ 0000000180005308     libgc.obj
 0002:00001320       ??_C@_0BB@NOKBFPFO@java?1lang?1Thread@ 0000000180005320     libgc.obj
 0002:00001334       ??_C@_06FALKBLGB@?$DMinit?$DO@ 0000000180005334     libgc.obj
 0002:00001340       ??_C@_0BG@IKDDPPGD@?$CILjava?1lang?1String?$DL?$CJV@ 0000000180005340     libgc.obj
 0002:00001360       ??_C@_0EB@IFJBFEKC@?$CIthreadClass?5?$DN?5jni_env?9?$DOFindCla@ 0000000180005360     libgc.obj
 0002:000013b0       ??_C@_0GF@FGFIBKKL@?$CIthreadCtor?5?$DN?5jni_env?9?$DOGetMetho@ 00000001800053b0     libgc.obj
 0002:00001418       ??_C@_0DN@NCPDJLOG@?$CIthreadName?5?$DN?5jni_env?9?$DONewStrin@ 0000000180005418     libgc.obj
 0002:00001460       ??_C@_0FE@PFKODBGC@?$CIthreadObject?5?$DN?5jni_env?9?$DONewObj@ 0000000180005460     libgc.obj
 0002:000014c0       ??_C@_0ED@HOBAHHJI@?$CIthreadGlobalRef?5?$DN?5jni_env?9?$DONew@ 00000001800054c0     libgc.obj
 0002:00001510       ??_C@_0FN@HNJJAHFC@jvmti_env?9?$DORunAgentThread?$CIagent@ 0000000180005510     libgc.obj
 0002:00001570       ??_C@_0EA@MOJDNKDF@Debuggee?5status?5sync?5aborted?5be@ 0000000180005570     libgc.obj
 0002:000015b0       ??_C@_0EA@EEOEJAEN@status?5?$DN?5syncDebuggeeStatus?$CIjni@ 00000001800055b0     libgc.obj
 0002:000015f0       ??_C@_0BL@JBCFNBMB@nsk_jvmti_resetAgentData?$CI?$CJ@ 00000001800055f0     libgc.obj
 0002:00001610       ??_C@_0EL@LPBEELIP@s?2test?2hotspot?2jtreg?2vmTestbase@ 0000000180005610     libgc.obj
 0002:00001660       ??_C@_0CK@JDAMFDMJ@jvmti?9?$DOSetTag?$CIo?0?5tag?$CJ?5?$DN?$DN?5JVMTI_@ 0000000180005660     libgc.obj
 0002:00001690       ??_C@_0CC@DAMNHKNI@Can?8t?5set?5tag?5?$CFli?5for?5object?5?$CFl@ 0000000180005690     libgc.obj
 0002:000016b8       ??_C@_0DL@HAJPNKEF@jvmti?9?$DOGetObjectHashCode?$CIo?0?5?$CGha@ 00000001800056b8     libgc.obj
 0002:000016f8       ??_C@_0BL@JFPIEOBF@Can?8t?5get?5hash?5object?5?$CFlx?6@ 00000001800056f8     libgc.obj
 0002:00001718       ??_C@_0BG@DICPHBKN@setTag?3?5?$CF08x?5?$DM?9?5?$CF?53li@ 0000000180005718     libgc.obj
 0002:00001730       ??_C@_0DH@FCEEBDMJ@?$CIs?5?$DN?5jni?9?$DOGetStringUTFChars?$CIsIn@ 0000000180005730     libgc.obj
 0002:00001768       ??_C@_0BJ@OKKGHDCN@Can?8t?5get?5string?5at?5?$CF?$CDp?6@ 0000000180005768     libgc.obj
 0002:00001788       ??_C@_0BP@EKFLGGFJ@Can?8t?5get?5string?5at?5?$CF?$CDp?3?5null?6@ 0000000180005788     libgc.obj
 0002:000017a8       ??_C@_06ICODBHCL@?5?1?1?5?$CFs@ 00000001800057a8     libgc.obj
 0002:000017b0       ??_C@_0DB@KGFPLEGO@?$CIr?5?$DN?5jvmti?9?$DOGetTag?$CIo?0?5?$CGtag?$CJ?$CJ?5?$DN?$DN@ 00000001800057b0     libgc.obj
 0002:000017e8       ??_C@_0CO@PDAGBCGJ@Can?8t?5GetTag?5for?5object?5?$CFlx?4?5Re@ 00000001800057e8     libgc.obj
 0002:00001818       ??_C@_0CH@HPEODOHC@TEST_BUG?3?5Max?4?5number?5of?5refs?5r@ 0000000180005818     libgc.obj
 0002:00001840       ??_C@_0DI@PHFCABIM@?$CIr?5?$DN?5jvmti?9?$DOGetTag?$CIfrom?0?5?$CGtagFr@ 0000000180005840     libgc.obj
 0002:00001878       ??_C@_0DI@MDEGFNKD@TEST_BUG?3?5Can?8t?5GetTag?5for?5obje@ 0000000180005878     libgc.obj
 0002:000018b0       ??_C@_0DE@MLELJAHM@?$CIr?5?$DN?5jvmti?9?$DOGetTag?$CIto?0?5?$CGtagTo?$CJ?$CJ@ 00000001800058b0     libgc.obj
 0002:000018e8       ??_C@_0BE@EEKKELIK@VMInit?5event?5?5done?6@ 00000001800058e8     libgc.obj
 0002:00001900       ??_C@_0DA@JDIEHOA@?9?9?9?9?9?9?9?9?9?9?9?9?5JVMTI_EVENT_VM_DEA@ 0000000180005900     libgc.obj
 0002:00001930       ??_C@_0DA@LGGMCEHG@JVMTI_EVENT_GARBAGE_COLLECTION_@ 0000000180005930     libgc.obj
 0002:00001960       ??_C@_0DB@IDFMEDN@JVMTI_EVENT_GARBAGE_COLLECTION_@ 0000000180005960     libgc.obj
 0002:00001998       ??_C@_0BN@KEIDFCPP@Event?3?5JVMTI_EVENT_GC_START?6@ 0000000180005998     libgc.obj
 0002:000019b8       ??_C@_0BO@ONLEDDEF@Event?3?5JVMTI_EVENT_GC_FINISH?6@ 00000001800059b8     libgc.obj
 0002:000019d8       ??_C@_09OPJEJKBL@printdump@ 00000001800059d8     libgc.obj
 0002:000019e8       ??_C@_0CJ@KCDEKOCJ@Wrong?5result?5of?5a?5valid?5call?5to@ 00000001800059e8     libgc.obj
 0002:00001a18       ??_C@_0N@HJAMKMBE@_access_lock@ 0000000180005a18     libgc.obj
 0002:00001a30       ??_C@_0EF@CGIKBHFH@RawMonitorEnter?5in?5monitor_cont@ 0000000180005a30     libgc.obj
 0002:00001a78       ??_C@_03PMGGPEJJ@?$CFd?6@  0000000180005a78     libgc.obj
 0002:00001a80       ??_C@_0CB@NJBLABLF@SetEventCallbacks?5returned?5erro@ 0000000180005a80     libgc.obj
 0002:00001aa8       ??_C@_0DE@MEFKDHFM@SetEventNotificationMode?5for?5VM@ 0000000180005aa8     libgc.obj
 0002:00001ae0       ??_C@_0DL@KHAEEJDH@SetEventNotificationMode?5for?5vm@ 0000000180005ae0     libgc.obj
 0002:00001b20       ??_C@_0DF@MIHDIEAB@SetEventNotificationMode?5for?5gc@ 0000000180005b20     libgc.obj
 0002:00001b58       ??_C@_0DG@GODLLLCA@SetEventNotificationMode?5for?5gc@ 0000000180005b58     libgc.obj
 0002:00001b90       ??_C@_0DH@KOKPNHIO@Error?3?5JVMTI_EVENT_GARBAGE_COLL@ 0000000180005b90     libgc.obj
 0002:00001bc8       ??_C@_0DI@CNHELMDA@Error?3?5JVMTI_EVENT_GARBAGE_COLL@ 0000000180005bc8     libgc.obj
 0002:00001c00       ??_C@_0BL@HLENPHJM@jvmti?5Force?5gc?5requested?5?6@ 0000000180005c00     libgc.obj
 0002:00001c20       ??_C@_0CD@FAOAJHGL@Error?3?5ForceGarbageCollection?5?$CF@ 0000000180005c20     libgc.obj
 0002:00001c60       ??_C@_1EC@JIJBPKFM@?$AAa?$AAp?$AAi?$AA?9?$AAm?$AAs?$AA?9?$AAw?$AAi?$AAn?$AA?9?$AAc?$AAo?$AAr?$AAe@ 0000000180005c60     MSVCRT:thread_safe_statics.obj
 0002:00001ca8       ??_C@_1BK@MGMFAEKH@?$AAk?$AAe?$AAr?$AAn?$AAe?$AAl?$AA3?$AA2?$AA?4?$AAd?$AAl?$AAl@ 0000000180005ca8     MSVCRT:thread_safe_statics.obj
 0002:00001cc8       ??_C@_0BJ@JEBJOJFJ@SleepConditionVariableCS@ 0000000180005cc8     MSVCRT:thread_safe_statics.obj
 0002:00001ce8       ??_C@_0BJ@PGPPEPCC@WakeAllConditionVariable@ 0000000180005ce8     MSVCRT:thread_safe_statics.obj
 0002:00001d08       _pDefaultRawDllMain        0000000180005d08     MSVCRT:dll_dllmain.obj
 0002:00001d08       _pRawDllMain               0000000180005d08     MSVCRT:dll_dllmain.obj
 0002:00001d10       __xmm@ffffffffffffffffffffffffffffffff 0000000180005d10     MSVCRT:utility.obj
 0002:00001d20       _load_config_used          0000000180005d20     MSVCRT:loadcfg.obj
 0002:00001f00       _tls_used                  0000000180005f00     MSVCRT:tlssup.obj
 0002:00001f28       __volatile_metadata        0000000180005f28     <linker-defined>
 0002:000022e0       __rtc_iaa                  00000001800062e0     MSVCRT:initsect.obj
 0002:000022e8       __rtc_izz                  00000001800062e8     MSVCRT:initsect.obj
 0002:000022f0       __rtc_taa                  00000001800062f0     MSVCRT:initsect.obj
 0002:000022f8       __rtc_tzz                  00000001800062f8     MSVCRT:initsect.obj
 0002:00002300       _tls_start                 0000000180006300     MSVCRT:tlssup.obj
 0002:00002304       _Init_thread_epoch         0000000180006304     MSVCRT:thread_safe_statics.obj
 0002:00002308       _tls_end                   0000000180006308     MSVCRT:tlssup.obj
 0002:00002a84       __IMPORT_DESCRIPTOR_KERNEL32 0000000180006a84     kernel32:KERNEL32.dll
 0002:00002a98       __IMPORT_DESCRIPTOR_VCRUNTIME140 0000000180006a98     vcruntime:VCRUNTIME140.dll
 0002:00002aac       __IMPORT_DESCRIPTOR_api-ms-win-crt-runtime-l1-1-0 0000000180006aac     ucrt:api-ms-win-crt-runtime-l1-1-0.dll
 0002:00002ac0       __IMPORT_DESCRIPTOR_api-ms-win-crt-stdio-l1-1-0 0000000180006ac0     ucrt:api-ms-win-crt-stdio-l1-1-0.dll
 0002:00002ad4       __IMPORT_DESCRIPTOR_api-ms-win-crt-string-l1-1-0 0000000180006ad4     ucrt:api-ms-win-crt-string-l1-1-0.dll
 0002:00002ae8       __NULL_IMPORT_DESCRIPTOR   0000000180006ae8     kernel32:KERNEL32.dll
 0003:00000030       _Init_global_epoch         0000000180008030     MSVCRT:thread_safe_statics.obj
 0003:00000040       __security_cookie          0000000180008040     MSVCRT:gs_cookie.obj
 0003:00000048       __security_cookie_complement 0000000180008048     MSVCRT:gs_cookie.obj
 0003:00000050       __scrt_native_dllmain_reason 0000000180008050     MSVCRT:utility.obj
 0003:00000058       __isa_available            0000000180008058     MSVCRT:cpu_disp.obj
 0003:0000005c       __isa_enabled              000000018000805c     MSVCRT:cpu_disp.obj
 0003:00000060       __memset_fast_string_threshold 0000000180008060     MSVCRT:cpu_disp.obj
 0003:00000068       __memset_nt_threshold      0000000180008068     MSVCRT:cpu_disp.obj
 0003:00000070       __scrt_ucrt_dll_is_in_use  0000000180008070     MSVCRT:ucrt_stubs.obj
 0003:00000080       g_wrongHeapCallbacks       0000000180008080     libgc.obj
 0003:00000100       g_szTagInfo                0000000180008100     libgc.obj
 0003:00002040       g_tagFlags                 000000018000a040     libgc.obj
 0003:00002428       g_refsToVerifyCnt          000000018000a428     libgc.obj
 0003:0000242c       g_fakeUserData             000000018000a42c     libgc.obj
 0003:00002430       g_tagVisitCount            000000018000a430     libgc.obj
 0003:000033d0       g_refsToVerify             000000018000b3d0     libgc.obj
 0003:0001aad0       g_userDataError            0000000180022ad0     libgc.obj
 0003:0001aad4       iGlobalStatus              0000000180022ad4     libgc.obj
 0003:0001aad8       access_lock                0000000180022ad8     libgc.obj
 0003:0001aae0       jvmti                      0000000180022ae0     libgc.obj
 0003:0001aae8       printdump                  0000000180022ae8     libgc.obj
 0003:0001aaec       gc_start_count             0000000180022aec     libgc.obj
 0003:0001aaf0       susp_thrd                  0000000180022af0     libgc.obj
 0003:0001ab30       gc_finish_count            0000000180022b30     libgc.obj
 0003:0001ae18       ?_OptionsStorage@?1??__local_stdio_printf_options@@9@4_KA 0000000180022e18     libgc.obj
 0003:0001b3d8       _tls_index                 00000001800233d8     MSVCRT:tlssup.obj
 0003:0001b3e0       __scrt_current_native_startup_state 00000001800233e0     MSVCRT:utility.obj
 0003:0001b3e8       __scrt_native_startup_lock 00000001800233e8     MSVCRT:utility.obj
 0003:0001b428       __scrt_debugger_hook_flag  0000000180023428     MSVCRT:utility_desktop.obj
 0003:0001b430       ?__type_info_root_node@@3U__type_info_node@@A 0000000180023430     MSVCRT:tncleanup.obj
 0003:0001b440       ?_OptionsStorage@?1??__local_stdio_scanf_options@@9@4_KA 0000000180023440     MSVCRT:default_local_stdio_options.obj
 0003:0001b448       __favor                    0000000180023448     MSVCRT:cpu_disp.obj
 0003:0001b450       __dyn_tls_init_callback    0000000180023450     <common>

 entry point at        0001:00002410

 Static symbols

 0000:fffda000       .debug$S                   0000000180000000     gc.exp
 0000:fffda000       .debug$S                   0000000180000000     vcruntime:VCRUNTIME140.dll
 0000:fffda000       .debug$S                   0000000180000000     vcruntime:VCRUNTIME140.dll
 0000:fffda000       .debug$S                   0000000180000000     vcruntime:VCRUNTIME140.dll
 0000:fffda000       .debug$S                   0000000180000000     vcruntime:VCRUNTIME140.dll
 0000:fffda000       .debug$S                   0000000180000000     vcruntime:VCRUNTIME140.dll
 0000:fffda000       .debug$S                   0000000180000000     vcruntime:VCRUNTIME140.dll
 0000:fffda000       .debug$S                   0000000180000000     vcruntime:VCRUNTIME140.dll
 0000:fffda000       .debug$S                   0000000180000000     vcruntime:VCRUNTIME140.dll
 0000:fffda000       .debug$S                   0000000180000000     ucrt:api-ms-win-crt-convert-l1-1-0.dll
 0002:ffffc000       .idata$6                   0000000180000000     ucrt:api-ms-win-crt-convert-l1-1-0.dll
 0000:fffda000       .debug$S                   0000000180000000     ucrt:api-ms-win-crt-heap-l1-1-0.dll
 0000:fffda000       .debug$S                   0000000180000000     ucrt:api-ms-win-crt-heap-l1-1-0.dll
 0000:fffda000       .debug$S                   0000000180000000     ucrt:api-ms-win-crt-heap-l1-1-0.dll
 0000:fffda000       .debug$S                   0000000180000000     ucrt:api-ms-win-crt-heap-l1-1-0.dll
 0002:ffffc000       .idata$6                   0000000180000000     ucrt:api-ms-win-crt-heap-l1-1-0.dll
 0000:fffda000       .debug$S                   0000000180000000     ucrt:api-ms-win-crt-runtime-l1-1-0.dll
 0000:fffda000       .debug$S                   0000000180000000     ucrt:api-ms-win-crt-runtime-l1-1-0.dll
 0000:fffda000       .debug$S                   0000000180000000     ucrt:api-ms-win-crt-runtime-l1-1-0.dll
 0000:fffda000       .debug$S                   0000000180000000     ucrt:api-ms-win-crt-runtime-l1-1-0.dll
 0000:fffda000       .debug$S                   0000000180000000     ucrt:api-ms-win-crt-runtime-l1-1-0.dll
 0000:fffda000       .debug$S                   0000000180000000     ucrt:api-ms-win-crt-runtime-l1-1-0.dll
 0000:fffda000       .debug$S                   0000000180000000     ucrt:api-ms-win-crt-runtime-l1-1-0.dll
 0000:fffda000       .debug$S                   0000000180000000     ucrt:api-ms-win-crt-runtime-l1-1-0.dll
 0000:fffda000       .debug$S                   0000000180000000     ucrt:api-ms-win-crt-runtime-l1-1-0.dll
 0000:fffda000       .debug$S                   0000000180000000     ucrt:api-ms-win-crt-runtime-l1-1-0.dll
 0000:fffda000       .debug$S                   0000000180000000     ucrt:api-ms-win-crt-runtime-l1-1-0.dll
 0000:fffda000       .debug$S                   0000000180000000     ucrt:api-ms-win-crt-runtime-l1-1-0.dll
 0000:fffda000       .debug$S                   0000000180000000     ucrt:api-ms-win-crt-runtime-l1-1-0.dll
 0000:fffda000       .debug$S                   0000000180000000     ucrt:api-ms-win-crt-runtime-l1-1-0.dll
 0000:fffda000       .debug$S                   0000000180000000     ucrt:api-ms-win-crt-runtime-l1-1-0.dll
 0000:fffda000       .debug$S                   0000000180000000     ucrt:api-ms-win-crt-runtime-l1-1-0.dll
 0000:fffda000       .debug$S                   0000000180000000     ucrt:api-ms-win-crt-stdio-l1-1-0.dll
 0000:fffda000       .debug$S                   0000000180000000     ucrt:api-ms-win-crt-stdio-l1-1-0.dll
 0000:fffda000       .debug$S                   0000000180000000     ucrt:api-ms-win-crt-stdio-l1-1-0.dll
 0000:fffda000       .debug$S                   0000000180000000     ucrt:api-ms-win-crt-stdio-l1-1-0.dll
 0000:fffda000       .debug$S                   0000000180000000     ucrt:api-ms-win-crt-stdio-l1-1-0.dll
 0000:fffda000       .debug$S                   0000000180000000     ucrt:api-ms-win-crt-stdio-l1-1-0.dll
 0000:fffda000       .debug$S                   0000000180000000     ucrt:api-ms-win-crt-stdio-l1-1-0.dll
 0000:fffda000       .debug$S                   0000000180000000     ucrt:api-ms-win-crt-stdio-l1-1-0.dll
 0000:fffda000       .debug$S                   0000000180000000     ucrt:api-ms-win-crt-stdio-l1-1-0.dll
 0000:fffda000       .debug$S                   0000000180000000     ucrt:api-ms-win-crt-stdio-l1-1-0.dll
 0000:fffda000       .debug$S                   0000000180000000     ucrt:api-ms-win-crt-string-l1-1-0.dll
 0000:fffda000       .debug$S                   0000000180000000     ucrt:api-ms-win-crt-string-l1-1-0.dll
 0000:fffda000       .debug$S                   0000000180000000     ucrt:api-ms-win-crt-string-l1-1-0.dll
 0000:fffda000       .debug$S                   0000000180000000     ucrt:api-ms-win-crt-string-l1-1-0.dll
 0000:fffda000       .debug$S                   0000000180000000     ucrt:api-ms-win-crt-string-l1-1-0.dll
 0000:fffda000       .debug$S                   0000000180000000     ucrt:api-ms-win-crt-string-l1-1-0.dll
 0000:fffda000       .debug$S                   0000000180000000     ucrt:api-ms-win-crt-string-l1-1-0.dll
 0000:fffda000       .debug$S                   0000000180000000     ucrt:api-ms-win-crt-string-l1-1-0.dll
 0000:fffda000       .debug$S                   0000000180000000     kernel32:KERNEL32.dll
 0000:fffda000       .debug$S                   0000000180000000     kernel32:KERNEL32.dll
 0000:fffda000       .debug$S                   0000000180000000     kernel32:KERNEL32.dll
 0000:fffda000       .debug$S                   0000000180000000     kernel32:KERNEL32.dll
 0000:fffda000       .debug$S                   0000000180000000     kernel32:KERNEL32.dll
 0000:fffda000       .debug$S                   0000000180000000     kernel32:KERNEL32.dll
 0000:fffda000       .debug$S                   0000000180000000     kernel32:KERNEL32.dll
 0000:fffda000       .debug$S                   0000000180000000     kernel32:KERNEL32.dll
 0000:fffda000       .debug$S                   0000000180000000     kernel32:KERNEL32.dll
 0000:fffda000       .debug$S                   0000000180000000     kernel32:KERNEL32.dll
 0000:fffda000       .debug$S                   0000000180000000     kernel32:KERNEL32.dll
 0000:fffda000       .debug$S                   0000000180000000     kernel32:KERNEL32.dll
 0000:fffda000       .debug$S                   0000000180000000     kernel32:KERNEL32.dll
 0000:fffda000       .debug$S                   0000000180000000     kernel32:KERNEL32.dll
 0000:fffda000       .debug$S                   0000000180000000     kernel32:KERNEL32.dll
 0000:fffda000       .debug$S                   0000000180000000     kernel32:KERNEL32.dll
 0000:fffda000       .debug$S                   0000000180000000     kernel32:KERNEL32.dll
 0000:fffda000       .debug$S                   0000000180000000     kernel32:KERNEL32.dll
 0000:fffda000       .debug$S                   0000000180000000     kernel32:KERNEL32.dll
 0000:fffda000       .debug$S                   0000000180000000     kernel32:KERNEL32.dll
 0000:fffda000       .debug$S                   0000000180000000     kernel32:KERNEL32.dll
 0000:fffda000       .debug$S                   0000000180000000     kernel32:KERNEL32.dll
 0000:fffda000       .debug$S                   0000000180000000     kernel32:KERNEL32.dll
 0000:fffda000       .debug$S                   0000000180000000     kernel32:KERNEL32.dll
 0000:fffda000       .debug$S                   0000000180000000     kernel32:KERNEL32.dll
 0000:fffda000       .debug$S                   0000000180000000     kernel32:KERNEL32.dll
 0000:fffda000       .debug$S                   0000000180000000     kernel32:KERNEL32.dll
 0000:fffda000       .debug$S                   0000000180000000     kernel32:KERNEL32.dll
 0001:00000f08       addRefToVerify             0000000180001f08 f   libgc.obj
 0001:00000f74       agentThreadWrapper         0000000180001f74 f   libgc.obj
 0001:000011c0       file_basename              00000001800021c0 f   libgc.obj
 0001:000018ac       startAgentThreadWrapper    00000001800028ac f   libgc.obj
 0001:00001bec       syncDebuggeeStatus         0000000180002bec f   libgc.obj
 0001:00001ed0       capture_previous_context   0000000180002ed0 f   MSVCRT:gs_report.obj
 0001:00001f44       ?__scrt_initialize_thread_safe_statics@@YAHXZ 0000000180002f44 f   MSVCRT:thread_safe_statics.obj
 0001:00002014       ?__scrt_uninitialize_thread_safe_statics@@YAXXZ 0000000180003014 f   MSVCRT:thread_safe_statics.obj
 0001:000020c0       $$000000                   00000001800030c0     MSVCRT:amdsecgs.obj
 0001:000020f0       ?dllmain_crt_dispatch@@YAHQEAUHINSTANCE__@@KQEAX@Z 00000001800030f0 f   MSVCRT:dll_dllmain.obj
 0001:00002140       ?dllmain_crt_process_attach@@YAHQEAUHINSTANCE__@@QEAX@Z 0000000180003140 f   MSVCRT:dll_dllmain.obj
 0001:00002258       ?dllmain_crt_process_detach@@YAH_N@Z 0000000180003258 f   MSVCRT:dll_dllmain.obj
 0001:000022dc       ?dllmain_dispatch@@YAHQEAUHINSTANCE__@@KQEAX@Z 00000001800032dc f   MSVCRT:dll_dllmain.obj
 0001:00002cf0       $$000000                   0000000180003cf0     MSVCRT:guard_dispatch.obj
 0001:00002d10       $$000000                   0000000180003d10     MSVCRT:guard_xfg_dispatch.obj
 0001:00002d26       ?fin$0@?0??dllmain_crt_process_attach@@YAHQEAUHINSTANCE__@@QEAX@Z@4HA 0000000180003d26 f   MSVCRT:dll_dllmain.obj
 0001:00002d3d       ?fin$0@?0??dllmain_crt_process_detach@@YAH_N@Z@4HA 0000000180003d3d f   MSVCRT:dll_dllmain.obj
 0001:00002d56       ?fin$1@?0??dllmain_crt_process_detach@@YAH_N@Z@4HA 0000000180003d56 f   MSVCRT:dll_dllmain.obj
 0001:00002d6a       ?filt$0@?0??dllmain_dispatch@@YAHQEAUHINSTANCE__@@KQEAX@Z@4HA 0000000180003d6a f   MSVCRT:dll_dllmain.obj
 0001:00002da0       __scrt_is_nonwritable_in_current_image$filt$0 0000000180003da0 f   MSVCRT:utility.obj
 0002:000001e8       ?__scrt_initialize_tss_var@@3P6AHXZEA 00000001800041e8     MSVCRT:thread_safe_statics.obj
 0002:00000310       ?opcLengths@@3QBEB         0000000180004310     libgc.obj
 0002:00001c48       GS_ExceptionPointers       0000000180005c48     MSVCRT:gs_report.obj
 0002:00002310       $unwind$fprintf            0000000180006310     libgc.obj
 0002:0000231c       $unwind$printf             000000018000631c     libgc.obj
 0002:00002328       $unwind$?NewObject@JNIEnv_@@QEAAPEAV_jobject@@PEAV_jclass@@PEAU_jmethodID@@ZZ 0000000180006328     libgc.obj
 0002:00002328       $unwind$nsk_lcomplain      0000000180006328     libgc.obj
 0002:00002328       $unwind$nsk_ldisplay       0000000180006328     libgc.obj
 0002:00002330       $unwind$nsk_lvdisplay      0000000180006330     libgc.obj
 0002:00002330       $unwind$_RTC_Initialize    0000000180006330     MSVCRT:initsect.obj
 0002:00002330       $unwind$_RTC_Terminate     0000000180006330     MSVCRT:initsect.obj
 0002:00002330       $unwind$?__scrt_initialize_thread_safe_statics@@YAHXZ 0000000180006330     MSVCRT:thread_safe_statics.obj
 0002:0000233c       $unwind$nsk_lvcomplain     000000018000633c     libgc.obj
 0002:00002354       $unwind$nsk_ltrace         0000000180006354     libgc.obj
 0002:00002354       $unwind$__report_gsfailure 0000000180006354     MSVCRT:gs_report.obj
 0002:0000235c       $unwind$nsk_lvtrace        000000018000635c     libgc.obj
 0002:0000235c       $unwind$__raise_securityfailure 000000018000635c     MSVCRT:gs_report.obj
 0002:0000235c       $unwind$__scrt_initialize_crt 000000018000635c     MSVCRT:utility.obj
 0002:0000235c       $unwind$__scrt_initialize_onexit_tables 000000018000635c     MSVCRT:utility.obj
 0002:0000235c       $unwind$__scrt_release_startup_lock 000000018000635c     MSVCRT:utility.obj
 0002:0000235c       $unwind$__scrt_uninitialize_crt 000000018000635c     MSVCRT:utility.obj
 0002:0000235c       $unwind$_onexit            000000018000635c     MSVCRT:utility.obj
 0002:00002364       $unwind$nsk_lverify        0000000180006364     libgc.obj
 0002:00002374       $unwind$nsk_vprintf        0000000180006374     libgc.obj
 0002:00002384       $unwind$nsk_printf         0000000180006384     libgc.obj
 0002:0000238c       $unwind$?nsk_jni_lverify@@YAHHPEAUJNIEnv_@@HQEBDH1ZZ 000000018000638c     libgc.obj
 0002:000023a0       $unwind$?nsk_jni_check_exception@@YAHPEAUJNIEnv_@@QEBDH@Z 00000001800063a0     libgc.obj
 0002:000023bc       $unwind$Java_nsk_jvmti_unit_FollowReferences_FollowRefObjects_resetTags 00000001800063bc     libgc.obj
 0002:000023bc       $unwind$Java_nsk_jvmti_unit_functions_ForceGarbageCollection_gc_checkGCFinish 00000001800063bc     libgc.obj
 0002:000023bc       $unwind$Java_nsk_jvmti_unit_functions_ForceGarbageCollection_gc_checkGCStart 00000001800063bc     libgc.obj
 0002:000023bc       $unwind$Java_nsk_jvmti_unit_functions_ForceGarbageCollection_gc_jvmtiForceGC 00000001800063bc     libgc.obj
 0002:000023bc       $unwind$addRefToVerify     00000001800063bc     libgc.obj
 0002:000023bc       $unwind$init_callbacks     00000001800063bc     libgc.obj
 0002:000023bc       $unwind$nsk_jvmti_resetAgentData 00000001800063bc     libgc.obj
 0002:000023bc       $unwind$nsk_jvmti_setFailStatus 00000001800063bc     libgc.obj
 0002:000023bc       $unwind$vmExit             00000001800063bc     libgc.obj
 0002:000023bc       $unwind$__scrt_initialize_default_local_stdio_options 00000001800063bc     MSVCRT:default_local_stdio_options.obj
 0002:000023bc       $unwind$?dllmain_crt_dispatch@@YAHQEAUHINSTANCE__@@KQEAX@Z 00000001800063bc     MSVCRT:dll_dllmain.obj
 0002:000023bc       $unwind$DllMain            00000001800063bc     MSVCRT:dll_dllmain_stub.obj
 0002:000023bc       $unwind$__GSHandlerCheck   00000001800063bc     MSVCRT:gshandler.obj
 0002:000023bc       $unwind$?__scrt_uninitialize_thread_safe_statics@@YAXXZ 00000001800063bc     MSVCRT:thread_safe_statics.obj
 0002:000023bc       $unwind$__scrt_acquire_startup_lock 00000001800063bc     MSVCRT:utility.obj
 0002:000023bc       $unwind$__scrt_dllmain_after_initialize_c 00000001800063bc     MSVCRT:utility.obj
 0002:000023bc       $unwind$__scrt_dllmain_before_initialize_c 00000001800063bc     MSVCRT:utility.obj
 0002:000023bc       $unwind$__scrt_dllmain_crt_thread_attach 00000001800063bc     MSVCRT:utility.obj
 0002:000023bc       $unwind$__scrt_dllmain_crt_thread_detach 00000001800063bc     MSVCRT:utility.obj
 0002:000023bc       $unwind$__scrt_dllmain_uninitialize_c 00000001800063bc     MSVCRT:utility.obj
 0002:000023bc       $unwind$__scrt_dllmain_uninitialize_critical 00000001800063bc     MSVCRT:utility.obj
 0002:000023bc       $unwind$atexit             00000001800063bc     MSVCRT:utility.obj
 0002:000023c4       $unwind$nsk_jvmti_lverify  00000001800063c4     libgc.obj
 0002:000023d8       $unwind$exitOnError        00000001800063d8     libgc.obj
 0002:000023e8       $unwind$Java_nsk_share_jvmti_ArgumentHandler_getAgentOptionsString 00000001800063e8     libgc.obj
 0002:000023fc       $unwind$Java_nsk_jvmti_unit_FollowReferences_FollowRefObjects_getTag 00000001800063fc     libgc.obj
 0002:000023fc       $unwind$Java_nsk_share_jvmti_DebugeeClass_checkStatus 00000001800063fc     libgc.obj
 0002:000023fc       $unwind$agentThreadWrapper 00000001800063fc     libgc.obj
 0002:0000240c       $unwind$startAgentThreadWrapper 000000018000640c     libgc.obj
 0002:00002428       $unwind$syncDebuggeeStatus 0000000180006428     libgc.obj
 0002:00002428       $unwind$__scrt_dllmain_exception_filter 0000000180006428     MSVCRT:utility.obj
 0002:0000243c       $unwind$Java_nsk_share_jvmti_DebugeeClass_resetAgentData 000000018000643c     libgc.obj
 0002:00002444       $unwind$MA_checkStatus     0000000180006444     libgc.obj
 0002:00002458       $unwind$Java_nsk_jvmti_unit_FollowReferences_FollowRefObjects_setTag 0000000180006458     libgc.obj
 0002:00002470       $unwind$Java_nsk_jvmti_unit_FollowReferences_FollowRefObjects_addRefToVerify 0000000180006470     libgc.obj
 0002:0000248c       $unwind$Agent_Initialize   000000018000648c     libgc.obj
 0002:0000248c       $unwind$_DllMainCRTStartup 000000018000648c     MSVCRT:dll_dllmain.obj
 0002:0000249c       $unwind$debug_printf       000000018000649c     libgc.obj
 0002:000024a8       $unwind$capture_previous_context 00000001800064a8     MSVCRT:gs_report.obj
 0002:000024b4       $unwind$__GSHandlerCheckCommon 00000001800064b4     MSVCRT:gshandler.obj
 0002:000024c0       $xdatasym                  00000001800064c0     MSVCRT:amdsecgs.obj
 0002:000024c4       $unwind$?dllmain_crt_process_attach@@YAHQEAUHINSTANCE__@@QEAX@Z 00000001800064c4     MSVCRT:dll_dllmain.obj
 0002:00002500       $unwind$?fin$0@?0??dllmain_crt_process_attach@@YAHQEAUHINSTANCE__@@QEAX@Z@4HA 0000000180006500     MSVCRT:dll_dllmain.obj
 0002:00002500       $unwind$?fin$0@?0??dllmain_crt_process_detach@@YAH_N@Z@4HA 0000000180006500     MSVCRT:dll_dllmain.obj
 0002:00002500       $unwind$?fin$1@?0??dllmain_crt_process_detach@@YAH_N@Z@4HA 0000000180006500     MSVCRT:dll_dllmain.obj
 0002:00002508       $unwind$?dllmain_crt_process_detach@@YAH_N@Z 0000000180006508     MSVCRT:dll_dllmain.obj
 0002:0000255c       $unwind$?dllmain_dispatch@@YAHQEAUHINSTANCE__@@KQEAX@Z 000000018000655c     MSVCRT:dll_dllmain.obj
 0002:00002584       $unwind$?filt$0@?0??dllmain_dispatch@@YAHQEAUHINSTANCE__@@KQEAX@Z@4HA 0000000180006584     MSVCRT:dll_dllmain.obj
 0002:0000258c       $unwind$__scrt_is_nonwritable_in_current_image 000000018000658c     MSVCRT:utility.obj
 0002:000025ac       $unwind$__scrt_is_nonwritable_in_current_image$filt$0 00000001800065ac     MSVCRT:utility.obj
 0002:000025b4       $unwind$__scrt_fastfail    00000001800065b4     MSVCRT:utility_desktop.obj
 0002:000025c4       $unwind$__security_init_cookie 00000001800065c4     MSVCRT:gs_support.obj
 0002:000025d0       $unwind$__isa_available_init 00000001800065d0     MSVCRT:cpu_disp.obj
 0002:000025e0       $xdatasym                  00000001800065e0     MSVCRT:guard_dispatch.obj
 0002:000025e8       $xdatasym                  00000001800065e8     MSVCRT:guard_xfg_dispatch.obj
 0002:000025f0       .edata                     00000001800065f0     gc.exp
 0002:00002618       rgpv                       0000000180006618     gc.exp
 0002:00002660       rgszName                   0000000180006660     gc.exp
 0002:000026a8       rgwOrd                     00000001800066a8     gc.exp
 0002:000026cc       szName                     00000001800066cc     gc.exp
 0002:000026d3       $N00001                    00000001800066d3     gc.exp
 0002:000026e2       $N00002                    00000001800066e2     gc.exp
 0002:000026ef       $N00003                    00000001800066ef     gc.exp
 0002:00002734       $N00004                    0000000180006734     gc.exp
 0002:00002771       $N00005                    0000000180006771     gc.exp
 0002:000027b9       $N00006                    00000001800067b9     gc.exp
 0002:000027f9       $N00007                    00000001800067f9     gc.exp
 0002:00002836       $N00008                    0000000180006836     gc.exp
 0002:00002878       $N00009                    0000000180006878     gc.exp
 0002:000028be       $N00010                    00000001800068be     gc.exp
 0002:00002903       $N00011                    0000000180006903     gc.exp
 0002:00002948       $N00012                    0000000180006948     gc.exp
 0002:00002983       $N00013                    0000000180006983     gc.exp
 0002:000029b1       $N00014                    00000001800069b1     gc.exp
 0002:000029e2       $N00015                    00000001800069e2     gc.exp
 0002:00002a11       $N00016                    0000000180006a11     gc.exp
 0002:00002a40       $N00017                    0000000180006a40     gc.exp
 0002:00002a75       $N00018                    0000000180006a75     gc.exp
 0002:00002e82       .idata$6                   0000000180006e82     kernel32:KERNEL32.dll
 0002:00002ef0       .idata$6                   0000000180006ef0     vcruntime:VCRUNTIME140.dll
 0002:00003052       .idata$6                   0000000180007052     ucrt:api-ms-win-crt-runtime-l1-1-0.dll
 0002:00003074       .idata$6                   0000000180007074     ucrt:api-ms-win-crt-stdio-l1-1-0.dll
 0002:00003094       .idata$6                   0000000180007094     ucrt:api-ms-win-crt-string-l1-1-0.dll
 0003:00000000       ?codeAttributeName@@3PEBDEB 0000000180008000     libgc.obj
 0003:00000008       ?lineNumberAttributeName@@3PEBDEB 0000000180008008     libgc.obj
 0003:00000010       ?localVarAttributeName@@3PEBDEB 0000000180008010     libgc.obj
 0003:00000018       ?localVarTypeAttributeName@@3PEBDEB 0000000180008018     libgc.obj
 0003:00000020       ?stackMapAttributeName@@3PEBDEB 0000000180008020     libgc.obj
 0003:00000028       ?callBytes@@3PAEA          0000000180008028     libgc.obj
 0003:0000002c       ?allocBytes@@3PAEA         000000018000802c     libgc.obj
 0003:0001ab34       redefineAttempted          0000000180022b34     libgc.obj
 0003:0001ab38       nsk_context                0000000180022b38     libgc.obj
 0003:0001ab44       redefineSucceed            0000000180022b44     libgc.obj
 0003:0001ab48       agentFailed                0000000180022b48     libgc.obj
 0003:0001ab4c       currentAgentStatus         0000000180022b4c     libgc.obj
 0003:0001ab50       context                    0000000180022b50     libgc.obj
 0003:0001ac08       agentThread                0000000180022c08     libgc.obj
 0003:0001ac10       agentThreadProc            0000000180022c10     libgc.obj
 0003:0001ac18       agentThreadArg             0000000180022c18     libgc.obj
 0003:0001ac20       agent_data                 0000000180022c20     libgc.obj
 0003:0001ac30       jvmti_env                  0000000180022c30     libgc.obj
 0003:0001ac38       jvm                        0000000180022c38     libgc.obj
 0003:0001ac40       jni_env                    0000000180022c40     libgc.obj
 0003:0001ac48       checkStatus_func           0000000180022c48     libgc.obj
 0003:0001ac50       ?codeAttributeIndex@@3GA   0000000180022c50     libgc.obj
 0003:0001ac54       ?lineNumberAttributeIndex@@3GA 0000000180022c54     libgc.obj
 0003:0001ac58       ?localVarAttributeIndex@@3GA 0000000180022c58     libgc.obj
 0003:0001ac5c       ?localVarTypeAttributeIndex@@3GA 0000000180022c5c     libgc.obj
 0003:0001ac60       ?stackMapAttributeIndex@@3GA 0000000180022c60     libgc.obj
 0003:0001ac64       ?stackFrameOffset@@3GA     0000000180022c64     libgc.obj
 0003:0001ac68       ?mode@@3HA                 0000000180022c68     libgc.obj
 0003:0001ac6c       ?constantPoolSize@@3GA     0000000180022c6c     libgc.obj
 0003:0001ac70       ?orig@@3PEBEEB             0000000180022c70     libgc.obj
 0003:0001ac78       ?gen@@3PEAEEA              0000000180022c78     libgc.obj
 0003:0001ac80       ?inputPos@@3PEAEEA         0000000180022c80     libgc.obj
 0003:0001ac88       ?endPos@@3PEBEEB           0000000180022c88     libgc.obj
 0003:0001ac90       ?genPos@@3PEAEEA           0000000180022c90     libgc.obj
 0003:0001ac98       ?markPos@@3PEAEEA          0000000180022c98     libgc.obj
 0003:0001aca0       ?constantPool@@3PEAPEADEA  0000000180022ca0     libgc.obj
 0003:0001aca8       ?constantPoolCount@@3GA    0000000180022ca8     libgc.obj
 0003:0001acac       ?zeroBytes@@3PAEA          0000000180022cac     libgc.obj
 0003:0001acb0       ?codeLength@@3IA           0000000180022cb0     libgc.obj
 0003:0001acb8       ?map@@3PEAIEA              0000000180022cb8     libgc.obj
 0003:0001acc0       ?widening@@3PEACEA         0000000180022cc0     libgc.obj
 0003:0001acd0       callbacks                  0000000180022cd0     libgc.obj
 0003:0001ae08       jvmti_caps                 0000000180022e08     libgc.obj
 0003:0001ae20       GS_ExceptionRecord         0000000180022e20     MSVCRT:gs_report.obj
 0003:0001aec0       GS_ContextRecord           0000000180022ec0     MSVCRT:gs_report.obj
 0003:0001b390       ?g_tss_cv@@3U_RTL_CONDITION_VARIABLE@@A 0000000180023390     MSVCRT:thread_safe_statics.obj
 0003:0001b398       ?g_tss_event@@3PEAXEA      0000000180023398     MSVCRT:thread_safe_statics.obj
 0003:0001b3a0       ?g_tss_mutex@@3U_RTL_CRITICAL_SECTION@@A 00000001800233a0     MSVCRT:thread_safe_statics.obj
 0003:0001b3c8       ?g_sleep_condition_variable_cs@@3P6AHPEAU_RTL_CONDITION_VARIABLE@@PEAU_RTL_CRITICAL_SECTION@@K@ZEA 00000001800233c8     MSVCRT:thread_safe_statics.obj
 0003:0001b3d0       ?g_wake_all_condition_variable@@3P6AXPEAU_RTL_CONDITION_VARIABLE@@@ZEA 00000001800233d0     MSVCRT:thread_safe_statics.obj
 0003:0001b3dc       ?__proc_attached@@3HA      00000001800233dc     MSVCRT:dll_dllmain.obj
 0003:0001b3f0       ?is_initialized_as_dll@@3_NA 00000001800233f0     MSVCRT:utility.obj
 0003:0001b3f1       ?module_local_atexit_table_initialized@@3_NA 00000001800233f1     MSVCRT:utility.obj
 0003:0001b3f8       ?module_local_atexit_table@@3U_onexit_table_t@@A 00000001800233f8     MSVCRT:utility.obj
 0003:0001b410       ?module_local_at_quick_exit_table@@3U_onexit_table_t@@A 0000000180023410     MSVCRT:utility.obj
